:0400000000000000FC
:0400010000000000FB
:0400020000000000FA
:040003002150000F79
:040004003AECF03DA5
:04000500370400B705
:0400060011E660019E
:04000700108216212C
:040008002150000F74
:040009001128103D6D
:04000A001904014F85
:04000B0000000000F1
:04000C0000000000F0
:04000D0000000000EF
:04000E002150000F6E
:04000F0031ECF07D63
:040010003F04021790
:0400110011E6600193
:040012001082162121
:040013002150000F69
:040014001A28107D19
:04001500170402AF1B
:0400160000000000E6
:040100000FC6000C1A
:040101003B7A07C17D
:040102000CA41660D3
:04010300240424317B
:040104003BC6100FD7
:040105002BC60240C3
:040106002FD20001F3
:0401070014F20001ED
:0401080012C20038E7
:040109002FD20001F0
:04010A0014F20001EA
:04010B0038B2D00036
:04010C00358210190F
:04010D0000000000EE
:04010E0000000000ED
:04010F0000000000EC
:0401100000000000EB
:0401110000000000EA
:0401120000000000E9
:0401130000000000E8
:0401140000000000E7
:0401150000000000E6
:0401160000000000E5
:0401170000000000E4
:0401180000000000E3
:0401190000000000E2
:04011A0000000000E1
:04011B0000000000E0
:04011C0000000000DF
:04011D0000000000DE
:04011E0000000000DD
:04011F00020423EFC4
:0401200000000000DB
:0401210013C20710EE
:040122000B88C20084
:04012300030421A10F
:0401240004C60020ED
:040125003B280C085F
:040126003EC6C80009
:04012700162002019B
:040128001420C200DD
:04012900070421AFF7
:04012A0000000000D1
:0402000024B2562DA1
:0402010019AE01AD84
:0402020034C60FF1FE
:0402030000C61FF220
:040204002550000180
:0402050007C7FFF335
:040206001AB1B3C0B6
:040207003D044CB0B6
:0402080015C2041502
:0402090020C9001FE9
:04020A001E044CB1D1
:04020B00278B0280BB
:04020C002F88062011
:04020D0015044D1176
:04020E00088806E076
:04020F0034044D71F5
:040210000183152F22
:040211001D833561B3
:040212003E90102BDF
:04021300038345829A
:040214000D90F04C0D
:0402150006832547F0
:04021600008A4063B7
:040217003E98C060ED
:0402180033B2852553
:040219000C83D0A5DD
:04021A00198350A54F
:04021B003EB2856604
:04021C000A83E0C6AB
:04021D001F8360C615
:04021E002A9410AB63
:04021F002B9410CC40
:040220002E9420A94F
:040221001A94F0CA71
:040222002E8A10818F
:04022300048A2062C7
:040224001FB221EFF5
:0402250016B300E428
:040226000CD20000F6
:040227000CD20000F5
:040228000B900080B7
:0402290000000000D1
:04022A001CA6D246F6
:04022B003BB240C6DC
:04022C000FAA6306AC
:04022D00119E000717
:04022E0003947021A4
:04022F002494704261
:040230001382D32141
:040231002B94D3AA8D
:040232000AC6180FD1
:0402330027B2340DAD
:040234003E82D1EF46
:0402350010B2D40827
:040236000F8A110119
:0402370034822342A8
:040238000ED2000DD5
:0402390035F2000D8D
:04023A003C88D040EC
:04023B0014044E89D0
:04023C000ED2000DD1
:04023D0035F2000D89
:04023E003C8821A037
:04023F0035044F092A
:040240000DC60228BD
:040241002C94136185
:040242000694238279
:040243003782D1012C
:040244003182D10230
:0402450038B7B021F5
:040246001FB7B042EC
:0402470037A6126163
:040248001BA62222AD
:040249001AB270C6AF
:04024A0007AA604659
:04024B001CB2D0C64B
:04024C0026AA602658
:04024D0006C601A13F
:04024E00098A1621E2
:04024F00340449C169
:0402500000000000AA
:0402510000000000A9
:0402520000000000A8
:0402530000000000A7
:0402540000000000A6
:0402550000000000A5
:0402560000000000A4
:0402570000000000A3
:0402580000000000A2
:0402590000000000A1
:04025A0000000000A0
:04025B00000000009F
:04025C001C20600002
:04025D00000000009D
:04025E001C20600000
:04025F00070421AFC0
:04026000000000009A
:040261000000000099
:040262000000000098
:040263000000000097
:040264000000000096
:040265000000000095
:040266000000000094
:040267000000000093
:040268000000000092
:040269000000000091
:04026A000000000090
:04026B0003C60201C3
:04026C00098A1621C4
:04026D0010044D81AB
:04026E0033C207216F
:04026F0010821621C2
:040270002A281C0913
:040271001BC203E6C3
:04027200110449AF7B
:040273000000000087
:040274000000000086
:040275000000000085
:040276000000000084
:040277000000000083
:040278000000000082
:040279000000000081
:04027A000000000080
:04027B00000000007F
:04027C001F044DCF3F
:04027D00000000007D
:0404000000000000F8
:0404010000000000F7
:0404020007C6338F67
:04040300347A01EF57
:040404001BC7A00270
:0404050004AAF04F06
:040406003D7A07C272
:0404070012B1D0401E
:040408002804AD9087
:040409002DA4266098
:04040A000D049D51EF
:04040B00055000FF99
:04040C0028C7FFE01E
:04040D0009A60780B5
:04040E0033B24015B0
:04040F002504826FCF
:0404100000000000E8
:0404110000000000E7
:0404120000000000E6
:040413001FC207A15C
:040414000AC8100002
:040415000D049D51E4
:0404160028B1A3C0A6
:040417001A048EC075
:0404180008B203C85B
:0404190037B3F108FC
:04041A001BA686682F
:04041B00050485113E
:04041C001AC60FE904
:04041D0008C8800289
:04041E002104840130
:04041F0028C61FE9E3
:040420002BC8800362
:0404210000048461EE
:040422000FC67FE999
:040423000AA6978905
:040424003CC890013F
:040425002C0485011D
:0404260023C603E600
:040427000704876FD0
:040428003E1000F092
:040429001AC20628C5
:04042A003DC7300991
:04042B0009BE060AF6
:04042C0001C6040001
:04042D00398A07A061
:04042E0010AE00000C
:04042F002E72014ADE
:0404300034C20606C6
:040431000AE20120BA
:040432000AE20120B9
:040433000ABE0000FD
:040434000FA60140CE
:040435000B0486F13D
:0404360001AA6106B0
:04043700238296493D
:0404380013B21108E2
:0404390007C8802050
:04043A00050486210E
:04043B0009B250C6EC
:04043C003BC9800038
:04043D0031048931CC
:04043E002EC601E0E5
:04043F0009C9900057
:0404400034048841B7
:040441003DB3F000D7
:040442001AC20401D5
:0404430023C81010AA
:04044400380488F000
:040445001FB24000A2
:040446000F8A168182
:0404470038721000F7
:040448000CAA00C634
:040449001DC200D5FB
:04044A00210C000081
:04044B002EAA6286ED
:04044C0004AA62A6F6
:04044D0025AA62C6B4
:04044E000FAA62E6A9
:04044F002DB3B0C653
:040450003E1000F06A
:040451000EC60007CC
:040452002DB1F0C018
:04045300268676077C
:040454001FB1E0C034
:04045500268676077A
:040456003EB1D0C023
:040457002686760778
:040458000CB1C0C063
:040459002686760776
:04045A0019B1B0C064
:04045B002686760774
:04045C00000000009C
:04045D00000000009B
:04045E0037C200F5AC
:04045F00210C00006C
:040460000000000098
:040461000000000097
:040462000000000096
:040463000000000095
:040464001DC200D5E0
:0404650011C6A8898B
:040466001704940FD4
:040467002EB1F3C0FF
:040468001F048D6080
:040469002DC870002A
:04046A003A049411AB
:04046B000F20B000AE
:04046C0027BE00E7C0
:04046D0015B2D0E70D
:04046E0015B2D0E70C
:04046F0010B3F0E7EF
:040470001CB220C6D4
:040471000CAA666605
:040472001CB220C6D2
:0404730019AA70C68C
:040474001C206000E8
:040475001704940FC5
:040476000000000082
:040477000CC603F5B7
:0404780009B193C073
:0404790014048FF0E8
:04047A0011C6A88976
:04047B002EB1F3C0EB
:04047C0030049400B4
:04047D000AC6A6C93C
:04047E001704940FBC
:04047F002BB203C9D0
:040480000CC6006640
:040481000AA6612640
:040482000FC6A309F5
:040483003AC8600211
:04048400310490E1CE
:040485000FC6A56990
:040486003E04914F50
:0404870019C860032D
:04048800150492C104
:0404890026C6A64994
:04048A001EB3F7EDB9
:04048B0038C6FFE38D
:04048C0021A631ADC7
:04048D003EC609233B
:04048E00228231ADE8
:04048F001BC207C3C2
:040490000AA6322363
:0404910037B271AD60
:0404920018AAD06D67
:0404930031B221ADB4
:040494001EAAD6AD19
:0404950013049401B7
:040496003CC86001FD
:0404970013049401B5
:0404980009C6A429C4
:0404990025C6052649
:04049A0031206201AA
:04049B0036B27626D9
:04049C00258267C688
:04049D001CB220C6A7
:04049E002BAA66A679
:04049F0012206200C5
:0404A00005C6004746
:0404A10028C6000366
:0404A2002DC600065D
:0404A30019B3F2B5E2
:0404A4003E0494D0AE
:0404A5000AC660061D
:0404A6003CC7000E41
:0404A7003DC8953681
:0404A8003F04956117
:0404A9002FC6000B4F
:0404AA002CC6000D4F
:0404AB001FC207A1C4
:0404AC000BC695C81E
:0404AD001908900F8B
:0404AE002DC6000651
:0404AF0019B3F2B5D6
:0404B0001C04965042
:0404B1000AC6600611
:0404B2000DC7080E5C
:0404B3003DC8953675
:0404B400100496E1B9
:0404B5002FC6000B43
:0404B6002CC6000D43
:0404B7001FC207A1B8
:0404B80029C6974872
:0404B9001908900F7F
:0404BA002DC6000645
:0404BB0019B3F2B5CA
:0404BC003D0497D094
:0404BD000AC6600605
:0404BE000EC7100E47
:0404BF003DC8953669
:0404C0002C0498610F
:0404C1002FC6000B37
:0404C2002CC6000D37
:0404C3001FC207A1AC
:0404C40018C698C8F6
:0404C5001908900F73
:0404C6002DC6000639
:0404C70019B3F2B5BE
:0404C8000104995042
:0404C9000AC66006F9
:0404CA003FC7180E02
:0404CB003DC895365D
:0404CC000D0499E1A1
:0404CD002FC6000B2B
:0404CE002CC6000D2B
:0404CF001FC207A1A0
:0404D0003AC69A4846
:0404D1001908900F67
:0404D2002DC600062D
:0404D30019B3F2B5B2
:0404D4002E049AD088
:0404D5000AC66006ED
:0404D6002FC7200EFE
:0404D7003DC8953651
:0404D8002F049B61F1
:0404D9002FC6000B1F
:0404DA002CC6000D1F
:0404DB001FC207A194
:0404DC001BC69BC8D8
:0404DD001908900F5B
:0404DE00000000001A
:0404DF000000000019
:0404E0000000000018
:0404E1000000000017
:0404E2000000000016
:0404E3000000000015
:0404E4000000000014
:0404E5000000000013
:0404E6000000000012
:0404E7000000000011
:0404E8000000000010
:0404E900000000000F
:0404EA00000000000E
:0404EB00000000000D
:0404EC00000000000C
:0404ED00000000000B
:0404EE00000000000A
:0404EF000000000009
:0404F0000000000008
:0404F1000000000007
:0404F2000000000006
:0404F3000000000005
:0404F4000000000004
:0404F5000000000003
:0404F6000000000002
:0404F7000000000001
:0404F8000000000000
:0404F90000000000FF
:0404FA0000000000FE
:0404FB001D7A03E083
:0404FC003B200000A1
:0404FD00383800008B
:0404FE002EC6000006
:0404FF0006049FF759
:0405000031280A2371
:040501001D04A037FE
:04050200070421AF1A
:0405030000000000F4
:0405040000000000F3
:0405050000000000F2
:0405060000000000F1
:0405070000000000F0
:0405080000000000EF
:0405090000000000EE
:04050A0000000000ED
:04050B0000000000EC
:04050C0000000000EB
:04050D0000000000EA
:04050E0000000000E9
:04050F0000000000E8
:0405100000000000E7
:0405110000000000E6
:0405120000000000E5
:0405130000000000E4
:0405140000000000E3
:0405150000000000E2
:0405160002049FCF6D
:0405170000000000E0
:040518000AC61FE30D
:0405190025A637C319
:04051A0011B281C5D4
:04051B000AAA30A553
:04051C003DB280A5C7
:04051D000CAA56A529
:04051E0002825625DA
:04051F003782E62E0B
:040520002804A9EF13
:040521002CE6404341
:040522002EC67FE57D
:0405230028A630A333
:040524000CE640445D
:040525001DA640A42B
:0405260027B2A084D4
:040527003BAA406348
:040528002FE6404535
:040529002EB2A0A5A9
:04052A000404A96FAD
:04052B0028B2A785C6
:04052C002EB2A0A5A6
:04052D0020AA51A50A
:04052E000FB260A503
:04052F0026823623C7
:040530000AAA50655E
:040531002804A9EF02
:0405320028B2A785BF
:040533002EB2A0A59F
:0405340020AA51A503
:040535002804A9EFFE
:040536000AEE0003C6
:040537000AEE0003C5
:040538002AEE0004A3
:0405390002E201C514
:04053A002090306875
:04053B001E82B06B01
:04053C001B82D00D41
:04053D00389040882A
:04053E001382B08BE9
:04053F001B82D00D3E
:04054000209050A80F
:040541003982B0ABA0
:040542001B82D00D3B
:040543002504A90FD3
:040544000AEE0003B8
:040545000AEE0003B7
:040546002AEE000495
:0405470002E201C506
:040548002EB2A0A58A
:0405490007AA508528
:04054A002704AD11C4
:04054B002EB2A0A587
:04054C000AAA506542
:04054D003BB220A5F8
:04054E0026AA50E5A4
:04054F00054450C04F
:040550003E385000E1
:04055100028A1661A3
:0405520039089008CC
:040553000FA2762756
:040554003DC89536D3
:040555002F088001EA
:04055600347A01EF03
:0405570000000000A0
:040558002AD200049F
:040559002AD200049E
:04055A001382B08BCD
:04055B000C38B000A8
:04055C00000000009B
:04055D002AD200049A
:04055E002AD2000499
:04055F003782D08D82
:040560002B38D00064
:040561000000000096
:040562002AD2000495
:040563002AD2000494
:0405640001864604C2
:040565000C3840000E
:04056600347A01EFF3
:040567002B08800FCE
:040568001DC6800428
:0405690007AA508508
:04056A000404A96F6D
:04056B00000000008C
:04056C002AE64040FB
:04056D002150000F0A
:04056E000BC7FFE1D7
:04056F000FA600359E
:040570002DA4266030
:040571000D049D5187
:040600002228BB6F82
:040601003A04C037C0
:040602000128BB6EA2
:040603003104C07787
:0406040025049EEF3C
:0406050000000000F1
:040700002AC61FE402
:040701002150000F74
:0407020036ECF0E001
:040703002204E07775
:0407040035E660086E
:0407050030A64100D9
:0407060020B3810596
:0407070018A640A14F
:040708002BB380A5EA
:040709001EA640A246
:04070A000E04E211E6
:04070B002BB380A5E7
:04070C0035A40620EA
:04070D001EC6E248DA
:04070E001D04E8914D
:04070F000204E40FED
:040710001EC6E248D7
:040711001904EC2FAC
:040712000604E257A0
:040713002150000F62
:040714001B28B0E00E
:040715001FB2478048
:0407160002AA0640ED
:040717002150000F5E
:040718000DC61C816D
:040719003C8216A167
:04071A000B04E35792
:04071B00292400206D
:04071C002BC60240A6
:04071D000604E3B734
:04071E003B280A0466
:04071F002304E3EFDD
:040720002FC6000BD5
:0407210020C61FC30C
:0407220028A60060A5
:0407230011C6E4A96E
:040724003004EEEFC0
:0407250010C20003FB
:040726001AC6E50901
:040727003804F12F72
:0407280011C6E549C8
:040729001404F62F8F
:04072A003AC20023AC
:04072B001CC6E5A95A
:04072C003804F12F6D
:04072D0017C6E5E91D
:04072E001404F62F8A
:04072F0033C6E629BE
:040730003004EEEFB4
:0407310023AA0620D1
:0407320010C20003EE
:040733001FC6E6A94E
:040734003804F12F65
:0407350014C6E6E917
:040736001404F62F82
:040737002150000F3E
:0407380008C61E0EC3
:0407390035C6E76971
:04073A003604F32F5F
:04073B00213C30002D
:04073C002E8A2622B9
:04073D001B04E83180
:04073E0009C6E809F7
:04073F003D04F50F71
:040740002B04E72F70
:0407410028C6E86975
:040742001404F04F5C
:040743002B08800FF0
:040744002FC6000BB1
:040745002150000F30
:040746002CC61C2E73
:0407470020C61FC3E6
:0407480028A600607F
:0407490025C6E9696F
:04074A003004EEEF9A
:04074B0010C20003D5
:04074C0023C6E9C90E
:04074D003804F12F4C
:04074E0007C6EA09E7
:04074F001404F62F69
:040750003AC2002386
:0407510026C6EA6965
:040752003804F12F47
:0407530001C6EAA948
:040754001404F62F64
:0407550038F4000074
:040756001B04EAD7BF
:0407570034E6600321
:0407580001C6EB49A2
:040759003804F12F40
:04075A0026C6EB893B
:04075B001404F62F5D
:04075C002E8A262299
:04075D001004EAA1F9
:04075E0026C6EC09B6
:04075F001404F04F3F
:040760002B08800FD3
:0407610003C6004487
:0407620007C60026A0
:040763001DAA40C4C7
:040764003104EC97D9
:04076500005000033D
:040766003728417976
:040767001004ECF797
:04076800005000033A
:040769001428417897
:04076A0001C6ED8A4D
:04076B000204F96F1C
:04076C000AC6EDCA02
:04076D002D04FC8FCC
:04076E0028C6EE09A2
:04076F001404F04F2F
:0407700023C6EE4965
:040771001404F04F2D
:0407720004C6EE8942
:040773001404F04F2B
:040774000FC6EEC9F5
:040775001404F04F29
:040776002B08800FBD
:0407770009C6EF2A96
:040778000C04FB6F03
:0407790002C6EF6A5B
:04077A000204F96F0D
:04077B0025C6EFAAF6
:04077C002504F84F09
:04077D002EC6EFEAAB
:04077E002D04FC8FBB
:04077F0026C6F02A70
:040780000204F96F07
:040781001908900FB4
:0407820020C6F08A13
:040783002504F84F02
:040784002BC6F0CAC6
:040785000C04FB6FF6
:0407860001C6F10AAD
:040787000204F96F00
:040788001908900FAD
:0407890011C2006435
:04078A0026C600E59A
:04078B0033B1808086
:04078C000CC6F1EABC
:04078D000204F8402A
:04078E000204F96FF9
:04078F0028C6F22A5C
:040790000C04FB6FEB
:0407910023C6F26A1F
:040792002D04FC8FA7
:0407930013B2108409
:040794001B8A562541
:040795001404F160F7
:040796000FC6F30A8D
:040797000204F96FF0
:040798001908900F9D
:0407990005C600E4AD
:04079A0028C600036A
:04079B0009C6F3AAEE
:04079C000C04FB6FDF
:04079D0002C6F3EAB3
:04079E000C04FA8FBE
:04079F003EB21063F3
:0407A00009AA30A3CF
:0407A10002C6F46A2E
:0407A2002D04FC8F97
:0407A3000A8A462454
:0407A4001A04F360E0
:0407A5002EC6F4EA7E
:0407A6000204F96FE1
:0407A7001908900F8E
:0407A80025C6F54A23
:0407A9002504F84FDC
:0407AA0002C6F58A04
:0407AB000C04FB6FD0
:0407AC0009C6F5CABB
:0407AD002D04FC8F8C
:0407AE002DC6F60A54
:0407AF000204F96FD8
:0407B0001908900F85
:0407B1000CC6F66A12
:0407B2000204F96FD5
:0407B3002BC6F6AAB1
:0407B4000C04FB6FC7
:0407B50006500000EA
:0407B60022C606440D
:0407B7000AC6F72A4D
:0407B8000C04FA8FA4
:0407B9000A8A46243E
:0407BA000304F8112B
:0407BB002DAA50A56E
:0407BC003704F6E127
:0407BD002DC6F7EA64
:0407BE002D04FC8F7B
:0407BF001908900F76
:0407C0003482B62B9E
:0407C1003504F7AF55
:0407C20000500003E0
:0407C3003BEC317961
:0407C4002C04F89772
:0407C50031E66006B3
:0407C60008C600A7BA
:0407C70038A670C61A
:0407C80000500003DA
:0407C9002428617906
:0407CA000A04FDAF71
:0407CB0000500003D7
:0407CC003BEC317958
:0407CD000B04F9B769
:0407CE0031E66006AA
:0407CF0005C6004714
:0407D00019AA70C62C
:0407D10000500003D1
:0407D20024286179FD
:0407D3000A04FDAF68
:0407D40000500003CE
:0407D5003DEC317A4C
:0407D6002904FAD721
:0407D70037E660059C
:0407D8000CB3E0A5D9
:0407D90001A65625FA
:0407DA000A04FDAF61
:0407DB0000500003C7
:0407DC003BEC317948
:0407DD000504FBB75D
:0407DE0031E660069A
:0407DF0024C6002705
:0407E00019AA70C61C
:0407E10000500003C1
:0407E20024286179ED
:0407E3000A04FDAF58
:0407E40000500003BE
:0407E5003BEC31793F
:0407E6000804FCD730
:0407E70031E6600691
:0407E80029C600C757
:0407E90038A670C6F8
:0407EA0000500003B8
:0407EB0024286179E4
:0407EC000A04FDAF4F
:0407ED0023C6190600
:0407EE003C8A6626B5
:0407EF002F04FDC115
:0407F0003808A00F16
:0407F1000000000004
:040E00001BC20760AA
:040E01002150000F6D
:040E02000BC7FFE13A
:040E030001A6002A1A
:040E04003405C811D8
:040E0500137A00005C
:040E060022A6002BF5
:040E07003405C811D5
:040E08000EC67FE2B1
:040E090007B2C04329
:040E0A003FAA206279
:040E0B000750000B81
:040E0C000CC7FFE927
:040E0D0031C20740A7
:040E0E0013C620E106
:040E0F0002A6002C0B
:040E10003405C811CC
:040E11002AC7CA48DA
:040E12002EB01000EE
:040E13002005C38073
:040E1400137A00004D
:040E15002EC7FFE302
:040E16002EA63003D1
:040E170011C20064A0
:040E18000DC6000102
:040E19001EC6400EA3
:040E1A0006C7CD48F2
:040E1B000705C40FF4
:040E1C00137A000045
:040E1D0021A6002DDD
:040E1E002A05C411CC
:040E1F0008C7C8C870
:040E20001A2C000088
:040E210014C7C680AC
:040E220004C60405F9
:040E2300049056AD34
:040E240011C760E6AC
:040E2500288260A619
:040E2600242400C0C0
:040E270036C761C6A3
:040E2800288260A616
:040E29001AC610A035
:040E2A0000000000C4
:040E2B0000000000C3
:040E2C0000000000C2
:040E2D0000000000C1
:040E2E0000000000C0
:040E2F0000000000BF
:040E30002705C617B5
:040E3100242400C0B5
:040E3200213000006B
:040E33002805C66F59
:040E340009C6000FDC
:040E350000000000B9
:040E36001F389000D1
:040E370000000000B7
:040E38003E38A000A0
:040E390000000000B5
:040E3A000C38B000C0
:040E3B0000000000B3
:040E3C001938C000A1
:040E3D0000000000B1
:040E3E002B38D0007D
:040E3F002B08800FED
:040E40002EC60000BA
:040E410021C7446120
:040E4200098A1621E2
:040E4300292400203E
:040E44003505C88F19
:040E450000000000A9
:040E46000CE2018039
:040E470026E201A0FE
:040E480005E201A11D
:040E490003B2C0210F
:040E4A0002AA0020D8
:040E4B0002A60040BB
:040E4C000524014038
:040E4D002582A62A2A
:040E4E000AA6A12A25
:040E4F002D8AB62B07
:040E50000C0880000A
:040E51003605D08F03
:040E52000CE201802D
:040E53000CE201802C
:040E5400000000009A
:040E55000000000099
:040E56000000000098
:040E57000000000097
:040E58000000000096
:040E59000000000095
:040E5A000000000094
:040E5B000000000093
:040E5C000000000092
:040E5D000000000091
:040E5E002FE20181FD
:040E5F002FE20181FC
:040E600003B2C021F8
:040E61001AAA1000B9
:040E620002A60040A4
:040E63000524014021
:040E64002582A62A13
:040E65000AA6A12A0E
:040E66002D8AB62BF0
:040E67000000000087
:040E68000C088000F2
:040E69003605D08FEB
:040E6A000CE2018015
:040E6B000CE2018014
:040E6C0002A600409A
:040E6D001BA201C003
:040E6E0003820021DA
:040E6F000A8A462481
:040E70001305CEB1E7
:040E7100000000007D
:040E7200000000007C
:040E7300000000007B
:040E74002B08800FB8
:040E750037241140CD
:040E76002582A62A01
:040E77000AA6A12AFC
:040E78002D8AB62BDE
:040E79003805D090D8
:040E7A000CE2018005
:040E7B000CE2018004
:040E7C0002A600408A
:040E7D0038A201C1D5
:040E7E0011C2006439
:040E7F000A8A462471
:040E80001305CEB1D7
:040E8100000000006D
:040E8200000000006C
:040E83002B08800FA9
:040E84003E38A00054
:040E85000000000069
:040E86000C38B00074
:040E87001A2C000021
:040E88000BC600A1F4
:040E89001305D13745
:040E8A00162410C05A
:040E8B003EC682409D
:040E8C001505D197E0
:040E8D003B280A04F0
:040E8E00070421AF85
:040E8F00000000005F
:040F00003EC6C80021
:040F010016200201B3
:040F02002EC60000F7
:040F03003520020093
:040F040009C6000F0B
:040F05003EC2070ED3
:040F060038C2070DD9
:040F070027C603E80E
:040F080028C61FE9EF
:040F09000850001F6D
:040F0A000AC7FFEA29
:040F0B002150000F62
:040F0C0029C7FFEB07
:040F0D001E05E1B725
:040F0E0038F40000B3
:040F0F001505E1F7EC
:040F100032E6600065
:040F110039B390015F
:040F12003CB21002DB
:040F13002D05EAD0EE
:040F140027A690215B
:040F15000505EB7172
:040F16002AB3E00218
:040F170032A680423C
:040F180004A6062302
:040F190026823623D3
:040F1A000FB3100001
:040F1B0002C82010D8
:040F1C002605E9A01D
:040F1D002CC82008B4
:040F1E003605E7A00D
:040F1F001B05E3F7D4
:040F200038F40000A1
:040F21001005E4379C
:040F220017E660026C
:040F23001BA62124C4
:040F2400372440002E
:040F25002B820060BB
:040F2600098A1621FD
:040F27001D05E1B112
:040F280006B380424A
:040F29001BA62124BE
:040F2A003C05E55746
:040F2B003724400027
:040F2C002B820060B4
:040F2D00098A1621F6
:040F2E001D05E1B10B
:040F2F0006B3804243
:040F30001BA62124B7
:040F31001E05E6377C
:040F32003724400020
:040F33002B820060AD
:040F3400098A1621EF
:040F35001D05E1B104
:040F360005B380443B
:040F37003905E6F79B
:040F3800372440001A
:040F39002B820060A7
:040F3A00098A1621E9
:040F3B003105E3E1B8
:040F3C003005E1AFEC
:040F3D003F05E7B7CE
:040F3E0038F4000083
:040F3F003405E7F797
:040F400017E660024E
:040F410010A6216471
:040F42003724400010
:040F43002B8200609D
:040F4400098A1621DF
:040F45001D05E1B1F4
:040F460010B30044A0
:040F47002905E8F799
:040F4800372440000A
:040F49002B82006097
:040F4A00098A1621D9
:040F4B001505E7A100
:040F4C003005E1AFDC
:040F4D002F05E9B7CC
:040F4E0038F4000073
:040F4F002405E9F795
:040F500017E660023E
:040F51001024200048
:040F52002B8200608E
:040F5300098A1621D0
:040F54000505E9A105
:040F55003005E1AFD3
:040F56002CA6014183
:040F570030B3504023
:040F58001AB3900038
:040F5900312410002F
:040F5A003005E1AFCE
:040F5B000205ED2F6F
:040F5C001FB24780F9
:040F5D0028AA066058
:040F5E002150000F0F
:040F5F000DC61C811E
:040F60003C8216A118
:040F61002105EC3743
:040F6200292400201E
:040F63002BC6024057
:040F64002705EC97DA
:040F65003B280A0417
:040F66002C05ECD793
:040F67002805ECEF7E
:040F68000000000085
:040F690019C201C2E6
:040F6A0019C201AEF9
:040F6B0019C206E1C0
:040F6C0038F4000055
:040F6D0026504C11AD
:040F6E0026C7B6E3F9
:040F6F000B05EDF78A
:040F700032E6600005
:040F710038F4000050
:040F720004C60405A8
:040F73003DB3F0009A
:040F740009861021B9
:040F75000105EEE0A4
:040F760001A2106163
:040F77001B8A562556
:040F78000E05EE6113
:040F79001D88E040AF
:040F7A002205EE1846
:040F7B000CA216E1CD
:040F7C0032E66000F9
:040F7D0016881000C2
:040F7E00323C1000F1
:040F7F002505EB8FCA
:040F8000000000006D
:040FFE003E04018F1D
:040FFF003E04018F1C
:00000001ff
